:10190400566F6C746167652043616C6962000418EA
:1019140000000141444300000000000100000418DD
:1019240000000144656D616E640000010004013231
:1019340000000044697361626C65000100080418CA
:10194400000009444143000000000001000904189C
:101954000000094F4144430000000001000D045DF4
:101964000000094741444300000000010011000049
:0E197400000000000000000000000000000065
:0620C100019601011E0062
:101B5600E4F5D4F5D7F5D175A4BD7580FF75A59DBF
:101B66007590FFEF602B9000041205A7000000009F
:101B7600E4900008F0A31205A70000000090000DF5
:101B86001205A7000000009000111205A73F800073
:101B960000E4F51FD285D2927D0D7F03121E837D50
:101BA600037F01121E83E51EC454F0440FFD7F021D
:081BB600121E837F01021F5B78
:10200B0075D102E4F5BAEF540FF5BB75BCE0C2AF66
:10201B00C2EDD2EC30EDFDD2AF121D33AFBFEFFEF0
:04202B00ADBEEDFF5A
:01202F00228E
:03188000C9EFC9E4
:10188300C283E4FF7E08C284E95ED394004003D39D
:101893008001C39287D284EEC313FE0FBF04E7E433
:1018A300FF7E08C284ED5ED394004003D38001C35E
:1018B3009287D284EEC313FE0FBF04E7CFEACFCDE6
:1018C300EFCDE4FF7E80C284ED5ED394004003D36A
:1018D3008001C39287D284EEC313FE0FBF08E7EBE8
:1018E300FDE4FF7E80C284ED5ED394004003D38089
:1018F30001C39287D284EEC313FE0FBF08E7D283DE
:0119030022C1
:0416D300155D155D2F
:1016D700E4FFFEFDFC900009E0F8A3E0F9A3E0FABF
:1016E700A3E0FB1202C4500A9000091205A70000EC
:1016F7000000E4FFFE7D207C40900009E0F8A3E0B5
:10170700F9A3E0FAA3E0FB1202C4600C400A9000C0
:10171700091205A740200000E4FBFA7920784090E1
:101727000009E0FCA3E0FDA3E0FEA3E0FF1202270F
:101737007B007AFF797F784712011EE4FBFAF9787C
:101747003F12002D12036FA85DEEF608EFF6A85DB5
:0C175700E6FA08E6FB7D047F0312188010
:05176300055D055D229B
:101E8300C294E4FEC293C297D2930EBE04F6E4FE5C
:101E93007C08C293EF5CD394004003D38001C392C8
:101EA30097D293ECC313FC0EBE04E7D294C294E41E
:101EB300FE7C80C293ED5CD394004003D38001C3C6
:0E1EC3009297D293ECC313FC0EBE08E7D294A4
:011ED10022EE
:061AED008B5A8A5B895C44
:101AF300C294E4FEC293EEB40103D38001C3929770
:101B0300D2930EBE04EEE4FE7D08C293EF5DD39440
:101B1300004003D38001C39297D293EDC313FD0E0C
:101B2300BE04E7D294C294E4FE7D80AB5AAA5BA9BB
:101B33005C120436C29330960DAB5AAA5BA95C12B1
:101B430003F04D120436D293EDC313FD0EBE08E429
:021B5300D2942A
:011B5500226D
:0614F9008B3C8A3D893E98
:1014FF00C294E4F53FC293E53FB40103D38001C327
:10150F009297D293053FE53FB404EAE4F53F7E0896
:10151F00C293EF5ED394004003D38001C39297D25E
:10152F0093EEC313FE053FE53FB404E4D294C29497
:10153F00E4F53FAB3CAA3DA93E1205D800000000E0
:10154F00AB3CAA3DA93E12053578011205221205C2
:10155F0055C293AB3CAA3DA93EEBC0E0EAC0E0E91F
:10156F00C0E012056FA296E4334BFFEAFEE9FDE8F7
:10157F00FCD0E0F9D0E0FAD0E0FB120555D293058C
:08158F003FE53FB418BAD29405
:011597002231
:101450003095037F00227B007A0079347F041214D8
:10146000F9AF37AE36AD35AC34E4120331E4FBFAF4
:101470007980784B1202277B0A7AD7792378401239
:10148000011E8F3B8E3A8D398C387F007E507DC394
:101490007C47AB3BAA3AA939A83812011EE4FBFAF3
:1014A000F9783F12002D1212F57B007A5079C3783B
:1014B000471202278F3B8E3A8D398C3890000DE011
:1014C000F8A3E0F9A3E0FAA3E0FB120029900011D1
:1014D000E0F8A3E0F9A3E0FAA3E0FB12011E8F3BC2
:1014E0008E3A8D398C38C2AF90000012059BD2AF76
:0814F0007D6F7F02121E831FB5
:0114F80022D1
:101F5B00155DA85DEFF6A85DE6FFB40103E4F51F80
:101F6B00EFB4021CE51FD394024015900008E0600B
:101F7B000CE4FBFA7D047F0312188080031216D346
:031F8B00055D22CF
:0520CB008F2E7F0022B2
:101F8E008B2E8A2F89301203F0AB31AA32A933126D
:101F9E000436AB2EAA2FA930900001120409AB31E2
:0D1FAE00AA32A9339000011204487F0222DC
:101C1F00121450EF6058E51FC394065051900009FD
:101C2F00E0F8A3E0F9A3E0FAA3E0FBE8C0E0E9C025
:101C3F00E0EAC0E0EBC0E0900000E0F8A3E0F9A319
:101C4F00E0FAA3E0FBA3E0FCA3E0FDA3E0FEA3E02A
:101C5F00FF120029D0E0FBD0E0FAD0E0F9D0E0F895
:0F1C6F0012002D90000912059B1216D3051F229B
:0320C7000186008F
:100E3800E47886F612208275E104E4F5E275E34071
:100E480075A401F5A5F5A675A72075B16775B20853
:100E5800121CDAE4F535F5367D01AF36121FE405CC
:100E680036E53670020535C39401E535940040E84F
:100E7800E4F520C20BC208C20ED20AC20DC20C7819
:100E880086F6C2B57863F67861F618F67868F6F5EE
:100E980035F536746A2536F8E4F60536E536700217
:100EA80005356414453570EBE4F535F536747E2563
:100EB80036F8E4F60536E53670020535640845353A
:100EC80070EB7D08E4FF122030E47866F6785EF671
:100ED800785EE6FF75F010A42412F582E5F0341967
:100EE800F583E493FE786626F6EE6005785E068064
:100EF800DFEFD39400402A90191FE493FB74019309
:100F0800FA740293F974551204361203F0645560AA
:100F180002D20C74AA1204361203F064AA6002D238
:100F28000C121245EF6003021007C20A74FFF5089D
:100F3800F509F50AF50BE4F50CF50DFE7F10FDFB40
:100F48007A00790E120618753AFF753B19753C043C
:100F5800753D00753E107B007A00790E121E31E453
:100F6800F535F536E536C4F8540FC868FFE535C4DD
:100F780054F048FE74122FF58274193EF583E493F9
:100F8800607974162FF58274193EF583E49320E294
:100F98005FE4F534E534C37896965054E536C4F8E2
:100FA800540FC868FFE535C454F048FE74122FF595
:100FB8008274193EF583E493FD7C00C004C0057D6E
:100FC80000741F2FF58274193EF583E493FB7401B6
:100FD80093FA740293F97866E68534F0A4FFE92F52
:100FE800F9EA35F0FAD007D006120618053480A4BD
:100FF8000536E53670020535020F6C7F018004D294
:101008000AE4FF121B56E5EF30E30DD203786706BA
:10101800E6750C00F50D8004E47867F6E4F535F51F
:10102800367A007B967D03AF36121A000536E53610
:1010380070020535C39401E535940040E402000EC2
:0520D0007868E6FF2224
:0300230002115275
:10115200C0E0C0F0C083C082C0D075D000C000C063
:1011620001C002C003C004C005C006C00730992FE9
:10117200C2997861067961E778636670117861F6E1
:02118200D20990
:0811840075220A0000D522FBD0
:04118C00C2B5801157
:081190007522140000D522FBBA
:101198007861E6247EF8E6F59920980302122A2061
:1011A8009A07200B04C2988075C29A7860E60624D4
:1011B8006AF8A699C2987860E6FFB40113786AE6DF
:1011C800FE70057860F6805AEE540724027869F6B6
:1011D800EFB4020E7869E6B40908786BE62403795F
:1011E80069F77860E6FFB4140476008035EFC378B9
:1011F8006996402E7860E624FFFDE434FFFC7B000E
:101208007A00796A1217687860E62469F8E66F60F0
:0312180002800B46
:08121B007522140000D522FB2E
:1012230012075778607600D007D006D005D004D0D7
:1012330003D002D001D000D0D0D082D083D0F0D060
:02124300E03297
:101A79007868E6FF7866E68FF0A47C002525FFEC00
:101A890035F0FE786BE675F010A4241FF582E5F0B9
:101A99003419F583E493FB740193FA740293F98F73
:0D1AA900828E83120409FF7B007A007923EE
:101AB6008F2E8B2F8A308931EA494B60161203F03C
:101AC600FFE52EFD7C00120003AB2FAA30A931EFF3
:031AD600120436C1
:081AD9007532140000D532FB48
:0C1AE100852E991220AA3099FDC299228E
:08206C007863EFF6C209D2B55A
:08207400752E140000D52EFBAF
:06207C00787EE6F59922D2
:101ED200C9EFC9E964017028EDC39B40347896E6E6
:101EE200FFEB2FFFE433FEEDC39FEE6480F87480B6
:101EF20098501ED20BC3ED9B7868F6786276012269
:101F0200B90214ED6B700AD20B7868F67862760229
:081F120022C20BE47862F62202
:101BBE00C9EFC9BAFF15BBFF12ED6B7002EC6A706C
:101BCE0049D20B7868F67862E9F622E9640170254D
:101BDE00C3ED9BEC9A401C7896E62BFFE43AFEC3CD
:101BEE00ED9FEC9E500DD20BC3ED9B7868F678629C
:101BFE007601228015B90218ED6B7002EC6A700A3C
:101C0E00D20B7868F67862760222C20BE47862F61E
:011C1E0022A3
:10075700786AE6FF54F8F524EF1205F207A00907B7
:10076700AB0A07BA1007C31107D21207E51907F931
:100777001A081820081E2808B82909B63309E537CA
:100787000A08390A18410A21490A2A500A6E6109DA
:100797007C700A669800000A99786BE6FDE509FB0C
:1007A7007F018021786BE6FC08E6FDAB09AA087F8C
:1007B700018025D20B78627603020A99786BE6FDF1
:1007C700E50BFB7F02121ED2020A99786BE6FC0842
:1007D700E6FDAB0BAA0A7F02121BBE020A99786BD1
:1007E700E6FDE509FB7F01121ED2200B03020A99E1
:1007F7008016786BE6FC08E6FDAB09AA087F0112B4
:100807001BBE200B03020A99787E76787F01020AC5
:100817009675EF10020A99C2ACE4F523D2B5FB7ABC
:100827000079237F7F121AB67B007A0079237F181D
:10083700121AB67B007A0079237F04121AB6785E03
:10084700E6121AAF7B007A007923AF08121AB67B3B
:10085700007A007923AF09121AB67B007A00792350
:10086700AF0A121AB67B007A007923AF0B121AB6B9
:100877007B007A007923AF0C121AB67B007A0079D5
:1008870023AF0D121AB6E4F525740E2525F8E612E6
:100897001AAF0525E525C3941040EE7B007A007951
:0608A70000AF23121AB697
:0808AD00752D0A0000D52DFB9A
:1008B500020969786BE6FFC3785E9640030209700A
:1008C50075F010EFA42412F582E5F03419AF82F526
:1008D5002B8F2CC2ACE4F523D2B5FB7A0079237FAC
:1008E5007F121AB67B007A0079237F0D121AB6851E
:1008F5002C82852B83E493121AAF852C82852B835A
:10090500740193121AAF852C82852B83740293127E
:100915001AAF852C82852B83740393121AAF852C0D
:1009250082852B83740493121AAFE4F525E52C24F4
:1009350005F582E4352BF583E5822525F582E43539
:1009450083F583E493121AAF0525E525C394084082
:0C095500DC7B007A007900AF23121AB698
:08096100752D0A0000D52DFBE5
:10096900C2B5D2AC020A99787E7678E408F67F029D
:10097900020A9612209D788712058F787E767C78F8
:1009890087E6787FF67888E67880F67889E6788150
:10099900F6788AE67882F67C007D057B007A007914
:1009A9007E1217687883EFF67F06020A96786BE65F
:1009B900FFB4010B08E6F50808E6F509020A66EF37
:1009C900B40208786CE6F508020A66786BE6B403A7
:1009D9000808E6F50A08E6F50B020A66E4F525E5D6
:1009E90025C3786B965016746C2525F8E6FF740EAE
:1009F9002525F8C6EFC60525E525B410E2805E7AFF
:100A0900007B327D017868E6FF121A00020A9978A4
:100A19006BE624FF92028078786BE624FF920180CE
:100A29006F7868E66005752702800B200D0575272C
:100A3900038003752701787E767908A6277C007DD7
:100A4900027B007A00797E1217687880EFF67F03BF
:100A590012206CE52764017037D20E8002D2087823
:100A69008676F1802B7A007B327D017F00121A0095
:100A7900787E7679786BE6787FF67C007D027B005C
:100A89007A00797E1217687880EFF67F0312206C5E
:100A9900E52464A06003020C54786AE664A160034B
:100AA900020B7C08E6FFC3785E964003020C54757E
:100AB900F010EFA42412F582E5F03419F583E493DC
:100AC900F52775F010EFA42416F582E5F03419F531
:100AD90083E49330E22F1220CB8F27787E767F082C
:100AE900A627E5272402FDE433FC7B007A00797E02
:100AF90012176874802527F8EFF6E5272403FF12FB
:100B0900206C020C54786BE6FF1220CBC2ACE4F5E2
:100B190023D2B5E527D39406402B7B007A007923AD
:100B29007F7F121AB67B007A007923AF27121AB693
:100B3900E4F525E525C395275007121A790525807F
:100B4900F205278018E5272478121AAFE4F525E580
:100B590025C395275007121A79052580F27B007A5B
:080B6900007900AF23121AB657
:080B7100752D0A0000D52DFBD3
:100B7900020C50786AE664A26003020C54785EE6BF
:100B8900FF786BE6FEC39F4003020C5408E6FDC3E1
:100B99009F4003020C54EEC39D4003020C5418E617
:100BA900F525E4F527E525D3786C96501FAF251276
:100BB90020CB75F010E525A42412F582E5F034194F
:100BC900F583E4932527F527052580D9C2ACE4F5FB
:100BD90023D2B5FB7A0079237F7F121AB67B007A7C
:100BE900007923AF27121AB6786BE6F525E525D3E8
:100BF900786C96503FE4F52675F010E525A424128B
:100C0900F582E5F03419F583E493FFE526C39F5097
:100C19001F7868E6FF7866E68FF0A47C002526FF3A
:100C2900EC35F0FE75F010E525121A92052680C8FC
:0F0C3900052580B97B007A007900AF23121AB627
:080C4800752D0A0000D52DFBFB
:100C5000C2B5D2ACE52464587047FA7B327D017886
:100C600068E6FF121A0075310075320075337F7B1C
:100C7000007A00796B121F8E8F27E5272478787E03
:100C8000F6E5272401FDE433FC7B007A00797E122F
:100C90001768747F2527F8EFF6E5272402FF122056
:100CA0006CE52464806009E52464886003020E37E3
:100CB0007862E6B4010F7A007B327D017868E6FF46
:100CC000121A00801AE4F525E525C3789696500F90
:100CD0007A007B327D01AF25121A00052580E97864
:100CE0006AE65407F527B4070A75260108E6F527D2
:100CF000088005E4F526786BE6F5281527E528C376
:100D0000785E964003020E1575F010E528A42412B3
:100D1000F582E5F03419F583E493FFE527D39F408E
:100D2000028F277862E6B401097868E6F52AF5298A
:100D30008009E4F5297896E614F52A7868A62978DA
:100D400068E6D3952A4003020E09E4F525E525C39C
:100D500095274003020DFE75F010E528A42416F532
:100D600082E5F03419F583E49330E203020DF9755E
:100D7000F010E528A42413F582E5F03419F583E496
:100D8000936438701BE527D394044008E526252595
:100D9000246C802A7860E6C39525FF74682F801E36
:100DA00075F010E528A42412F582E5F03419F583D6
:100DB000E493FFC37860E69F252525262469F8E69D
:100DC000FD7868E6FF7866E68FF0A4FFE5257A00F7
:100DD0002FFFEA35F0FE75F010E528A4241FF582F8
:100DE000E5F03419F583E493FB740193FA740293EC
:100DF000F98F828E83ED1204480525020D4DAF2830
:100E0000121F5B786806020D3F7868A629E5246406
:100E1000887024800FE528B4FF1D786CE6F520E586
:100E200024B48813787E76787860E62469F8E678CA
:070E30007FF67F0212206C27
:010E37002298
:107000007886E664F160030275203009FDC2AF7531
:10701000FFDE75FFADE4F535F534209829E4F53948
:10702000F53A20981DC3E53A9488E5399413501237
:08703000753F0A0000D53FFB8B
:10703800053AE53A70E4053980E0B2B480D4859920
:1070480034C298E534641A60030270FFF539F53AE2
:0E70580020981DC3E53A9488E5399413501230
:08706600753F0A0000D53FFB55
:10706E00053AE53A70E4053980E030989F85993508
:10707E00C298E4F539F53A20981DC3E53A9488E5AF
:05708E003994135012BB
:08709300753F0A0000D53FFB28
:10709B00053AE53A70E4053980E020980302701A4E
:1070AB00859935C298E4F539F53A20981DC3E53A30
:0870BB009488E539941350128A
:0870C300753F0A0000D53FFBF8
:1070CB00053AE53A70E4053980E020980302701A1E
:0970DB00859935C298D2B5C2991D
:0870E400753F140000D53FFBCD
:0670EC007599783099FD52
:0870F200753F0A0000D53FFBC9
:1070FA00C2B5027512E5346450706EF539F53A205E
:0D710A00981DC3E53A9488E539941350129E
:08711700753F0A0000D53FFBA3
:10711F00053AE53A70E4053980E020980302701AC9
:09712F00859935C298D2B5C299C8
:08713800753F140000D53FFB78
:087140007599793099FDC2999F
:08714800753F140000D53FFB68
:087150007599013099FDC29907
:08715800753F140000D53FFB58
:06716000E4F5993099FDF1
:08716600753F0A0000D53FFB54
:0F716E00C2B5027512E5346401702FD2B5C29913
:08717D00753F140000D53FFB33
:087185007599783099FDC2995B
:08718D00753F140000D53FFB23
:06719500E4F5993099FDBC
:08719B00753F0A0000D53FFB1F
:1071A300C2B5027512E53464026003027252F53906
:1071B300F53A20981DC3E53A9488E53994135012A3
:0871C300753F0A0000D53FFBF7
:1071CB00053AE53A70E4053980E020980302701A1D
:1071DB00859935C298E4F536E53513B392B4E535A8
:1071EB0025E0FEC3E49400EE94705029E5357F0052
:1071FB0025E0FEC39460501DE5B654F04408F5B687
:10720B00758F038E3B8F3C853C828E83E4F053B6A7
:0C721B00F0F58F80037536FFD2B5C299E4
:08722700753F140000D53FFB88
:08722F007599783099FDC299B0
:08723700753F140000D53FFB78
:06723F008536993099FD2F
:08724500753F0A0000D53FFB74
:10724D00C2B5027512E5346403600302737BF53930
:10725D00F53A20981DC3E53A9488E53994135012F8
:08726D00753F0A0000D53FFB4C
:10727500053AE53A70E4053980E020980302701A72
:10728500859935C298E4F539F53A20981DC3E53A54
:087295009488E53994135012AE
:08729D00753F0A0000D53FFB1C
:1072A500053AE53A70E4053980E020980302701A42
:1072B500859937C298E5351392B4E53525E0FEC3C7
:1072C500E49400EE9470400302701AE5357D0025C4
:1072D500E0FCC39460400302701AE5B654F044081C
:1072E500F5B6758F01E53775F020A42DFFE5F03C67
:1072F500F53B8F3CE4F538E538C394205043E4F57D
:1073050039F53A20981DC3E53A9488E53994135028
:017315001265
:08731600753F0A0000D53FFBA2
:10731E00053AE53A70E4053980E020980302701AC8
:10732E00053CE53CAE3B7002053B14F5828E83E5D1
:10733E0099F0C298053880B653B6F0E4F58FD2B501
:02734E00C299E2
:08735000753F140000D53FFB5E
:087358007599783099FDC29986
:08736000753F140000D53FFB4E
:06736800E4F5993099FDE7
:08736E00753F0A0000D53FFB4A
:10737600C2B5027512E53464046003027417F53968
:10738600F53A20981DC3E53A9488E53994135012CE
:08739600753F0A0000D53FFB22
:10739E00053AE53A70E4053980E020980302701A48
:1073AE00859935C298E53525E0F53D753E00E4F545
:1073BE0036F539F53A053EE53EAE3D7002053D1413
:1073CE00F5828E83E4932536F536053AE53A70025A
:0E73DE0005397004E539640270DBD2B5C2993E
:0873EC00753F140000D53FFBC2
:0873F4007599783099FDC299EA
:0873FC00753F140000D53FFBB2
:067404008536993099FD68
:08740A00753F0A0000D53FFBAD
:10741200C2B5027512E5346405600302750AF539D6
:10742200F53A20981DC3E53A9488E5399413501231
:08743200753F0A0000D53FFB85
:10743A00053AE53A70E4053980E020980302701AAB
:10744A00859935C298E4F539F53A20981DC3E53A8D
:08745A009488E53994135012E7
:08746200753F0A0000D53FFB55
:10746A00053AE53A70E4053980E020980302701A7B
:09747A00859937C298D2B5C29978
:08748300753F140000D53FFB2A
:08748B0075997F3099FDC2994B
:08749300753F140000D53FFB1A
:10749B007599203099FDE53525E0FCE53775F02031
:1074AB00A42400FFE5F03CF53D8F3EE4F536F538BE
:0274BB00C29974
:0874BD00753F140000D53FFBF0
:1074C500853E82853D83E493F5993099FD053EE53A
:1074D5003EAE3D7002053D14F5828E83E49325365C
:0B74E500F5360538E538B420CDC2991B
:0874F000753F140000D53FFBBD
:0674F8008536993099FD74
:0874FE00753F0A0000D53FFBB9
:10750600C2B58008E534B4060375EF10E5346407A8
:0A751600600302701A7886F6D2AF07
:017520002248
:101D33001220AA200A0B7A007B327D017F00121A3F
:101D430000300C0B7A007B1E7D017F00121A0030DD
:101D53000817300D147A007B327D017868E6FF1294
:101D63001A00C2081213A5D20A300E08300D05C29C
:101D73000E127000122090E47B2C7A01F9F8C31242
:071D830005115002D20D22F0
:0B20B600120E38121D33121C1F80F8A0
:10104800005EBCE2613FDD83C29C7E20A3FD1F41A0
:101058009DC3217FFCA2401E5F01E3BD3E6082DC90
:10106800237D9FC1421CFEA0E1BF5D0380DE3C6280
:10107800BEE0025CDF81633D7C22C09E1D43A1FF70
:101088004618FAA427799BC584DA3866E5BB590760
:10109800DB856739BAE406581947A5FB7826C49A50
:1010A800653BD987045AB8E6A7F91B45C6987A2440
:1010B800F8A6441A99C7257B3A6486D85B05E7B930
:1010C8008CD2306EEDB3510F4E10F2AC2F7193CD20
:1010D800114FADF3702ECC92D38D6F31B2EC0E5010
:1010E800AFF1134DCE90722C6D33D18F0C52B0EE00
:1010F800326C8ED0530DEFB1F0AE4C1291CF2D73F0
:10110800CA947628ABF517490856B4EA6937D58BDF
:101118005709EBB536688AD495CB2977F4AA4816CF
:10112800E9B7550B88D6346A2B7597C94A14F6A8BF
:10113800742AC896154BA9F7B6E80A54D7896B35AF
:0A11480070B8DCEEF4F7FAFDFEFFCC
:10176800155D155DA85DECF608EDF6155D155D15C2
:101778005DA85DC6EBC608C6EAC608C6E9C6E55D4B
:0417880024FCF55DEB
:10178C00F80808E4F6A85DF608F6E55D2407F9A864
:10179C005DE6FE08E6FFC3099719E76480F8EE647E
:1017AC0080985037E55D2404F8CBE6CB08E6FA08C0
:1017BC00E6F98F828E83120409A85D080866FFE59E
:1017CC005D2403F8EFF6E690104893A85D0808F640
:1017DC00A85D0806E61870B20680AFA85D0808E69A
:0117EC00FFFD
:0717ED00E55D2409F55D2212
:07000300ED6F90104893FF20
:01000A0022D3
:10203000EF701E7598D0E589540F4420F58953C878
:10204000E1438E10ED90114793F58DD28ED2ACC244
:03205000BCD2AF50
:01205300226A
:101CDA00D2AFD2A9D2BBE589540F4401F589E4F504
:101CEA008E758CDBF58AD28CF54DF54CF54BF54AA1
:101CFA00F551F550F54FF54E754764FFEF25E02590
:101D0A00E02492F8E4F6EF25E025E02493F8E4F6DF
:101D1A00EF25E025E02494F8E4F6EF25E025E02419
:081D2A0095F8E4F60FBF01D4A7
:011D3200228E
:02163600155D40
:10163800A85DE4F6A85DE6FFC3940140030216D056
:10164800EF25E025E02495F8E6FFD394004052A862
:101658005DE625E025E02493F8E67045EF30E015D7
:10166800A85DE6FF25E025E02495F8E6D39401403F
:10167800047D0080067D01A85DE6FF121F1AA85DA3
:10168800E6FF25E025E02495F816E66014EF25E04E
:1016980025E02494F8E6FEEF25E025E02493F8EE13
:1016A800F6A85DE625E025E02493F8E6600116A893
:1016B8005DE6FF25E025E02495F8E670057D01123A
:0816C8001F1AA85D0602163C82
:0316D000055D2293
:03000B0002198255
:10198200C0E0C0F0C083C082C0D0E8C0E0E9C0E0DF
:10199200EAC0E0EBC0E0ECC0E0EDC0E0EEC0E0EF9A
:1019A200C0E0758CDCE54D2401F54DE4354CF54C79
:1019B200E4354BF54BE4354AF54AD54718E5512451
:1019C20001F551E43550F550E4354FF54FE4354E0D
:1019D200F54E754764121636122054D0E0FFD0E05F
:1019E200FED0E0FDD0E0FCD0E0FBD0E0FAD0E0F9A0
:0E19F200D0E0F8D0D0D082D083D0F0D0E03258
:101FE400155DA85DEDF6155DA85DEFF6A85DE6FF4D
:101FF400C39401500D08E6FEEF25E025E02492F895
:07200400EEF6055D055D220B
:101A0000155D155DA85DEAF608EBF6155DA85DEDC0
:101A1000F6155DA85DEFF6A85DE6FFC39401505290
:101A2000EF25E025E02495F8E67047A85DE6FB2564
:101A3000E025E02493F8E67039A85D08E625E00487
:101A4000FFA85DE6FA25E025E02495F8EFF6A85D0D
:101A50000808E6FE08E6FF7C007D0A12046AEA2513
:101A6000E025E02494F8EFF6EB25E025E02493F858
:091A7000E4F6E55D2404F55D22B5
:101F1A00155DA85DEDF6155DA85DEFF6A85DE6FF17
:101F2A00C39401501CEF25E025E02492F8E66011E5
:101F3A00A85D08E670047F0180027F00A85D08EFB3
:101F4A00F6A85DE6700608E624FF92B4055D055D15
:011F5A002264
:0C209000C2AFAF4DAE4CAD4BAC4AD2AF6E
:01209C002221
:0C209D00C2AFAF51AE50AD4FAC4ED2AF51
:0120A9002214
:0C20AA00E4F548F549300F0375FFA5224E
:10000E00D20FE4F548F54975FF0775FFA543B28099
:01001E0022BF
:0E208200C20FE4F548F54975FFDE75FFAD228B
:102054000549E54970020548300F0CC394E8E5488A
:082064009403500375FFA5224F
:041FBB008E528F5360
:101FBF00E4F554F555C3E5559553E5549552501432
:101FCF007FE87E03121DDF1220AA0555E55570E547
:041FDF00055480E144
:011FE30022DB
:041DDF008E568F5736
:101DE300D3E55794FAE5569400500AEFD394004094
:101DF3003C001F80F6855658855759D3E55994FA08
:101E0300E558940040157FFA7E00121DDF74062505
:101E130059F55974FF3558F55880E0D3E5579400C8
:0D1E2300E55694004007AF59AE58121DDF80
:011E3000228F
:081D8A008B3D8A3E893F8D402C
:101D92001220AAAB41AA42A9431204A02400FFE5E3
:101DA200F03460FE853D44853E45853F46E4FDEDC9
:101DB200C39540501BEF2DF582E43EF583E493ABCF
:101DC20044AA45A9468D827583001204480D80DF1E
:0D1DD200AB41AA42A943E48540F00204CBD6
:081598008B3A8A3B893C8D3D32
:1015A0007886E664F16003021635122082C2AFE548
:1015B000B654F04408F5B6758F01AB3EAA3FA9407A
:1015C0001204A02400FFE5F03460788BF608EFF6F3
:1015D000AA3BA93C788FA63A08C6EAC608C6E9C65F
:1015E000E4788DF6788DE6C3953D5032788FCBE662
:1015F000CB080806E618CAE6CA70010614F91203F9
:10160000F0788EF6E6FF788B0806E618CCE6CC700C
:10161000010614F5828C83EFF0788D0680C6E4F520
:101620008F53B6F0AB3EAA3FA940853DF01204CBE4
:05163000D2AF12000E14
:011635002292
:101C7E007886E664F17054C2AF122082E5B654F055
:101C8E004408F5B6758F03788D7660087600E47893
:101C9E008BF608F6788DE6FE08E6F5828E83E4F084
:101CAE001220AAE426F618740236F61806E6187004
:101CBE000106C3788CE6940818E66480948040D4BC
:0B1CCE00E4F58F53B6F0D2AF12000E09
:011CD90022E8
:1013A500121C7EE4F538F539F53E753F0075403879
:1013B500FB7A0079087D16121598E4F535E535C3F5
:1013C5007896965067E4F53475F010E534A4241248
:1013D500F582E5F03419F583E493604C7866E6858B
:1013E50035F0A4FFAEF075F010E534A4241FF582A6
:1013F500E5F03419F583E493FB740193FA740293D1
:101405002FF9EA3EFA75F010E534A42412F582E5C9
:10141500F03419F583E493FD753E00753F00754082
:1014250038121598053480A00535809175361275EA
:101435003734753E00753F007540387B007A00797A
:0A144500367D02121598E47886F651
:01144F00227A
:10124500E4F53BF53CF54175420075433BFB7A00FF
:1012550079087D16121D8AE4F538E538C378969627
:101265005067E4F53775F010E537A42412F582E5EB
:10127500F03419F583E493604C7866E68538F0A47C
:10128500FFAEF075F010E537A4241FF582E5F034C4
:1012950019F583E493FB740193FA7402932FF9EA29
:1012A5003EFA75F010E537A42412F582E5F03419FD
:1012B500F583E493FD75410075420075433B121DAE
:1012C5008A053780A0053880917541007542007503
:1012D500433B7B007A0079397D02121D8AE53A6429
:0F12E500347004E539641270047F0180027F00C9
:0112F40022D7
:100026000203DBE86480F8E933E83360110460F02A
:10003600ED33EC337009E8FCE9FDEAFEEBFF220440
:1000460060DED3EB9FEA9EE99DE8C2E78CF0C2F73B
:1000560095F0400CE8CCF8E9CDF9EACEFAEBCFFB07
:100066001203A685D0F05804700320D5B3E80470B7
:10007600075002B2D50203E592D5EC0460F7E4CC52
:10008600C0E0C398F8603B94186008400DD0E0FBD0
:100096000203BDE4FBFAC9FC8028E830E406E4C9A3
:1000A600FBE4CAFCE830E305E4C9CACBFCE8540724
:1000B6006010F8C3E913F9EA13FAEB13FBEC13FC2F
:1000C600D8F130F52FC3E49CFCEF9BFFEE9AFEEDD2
:1000D60099FDD0E0FBEF4E4D4C701222DB0302037C
:1000E600E2EC2CFCEF33FFEE33FEED33FDED30E7B3
:1000F600EB0203BDEF2BFFEE3AFEED39FDD0E0FB40
:1001060050130BBB00030203E5ED13FDEE13FEEFE8
:0801160013FFEC13FC0203BD12
:10011E00EC4D6011E8497017ED33EC3304600DE4DB
:10012E00FCFFFEFD22E933E8330470F80203DB1214
:10013E0003A658046009E4CC248150062850090215
:10014E0003E52840030203E2C0E0EB4A7044B980A5
:10015E0006D0E0FB0203D1EF4E701CBD8008EBFF12
:10016E00EAFEE9FD80EBE98DF0A4FEE5F002020760
:10017E00E9CDF9EAFEEBFFEF89F0A4FCE5F0CE89BC
:10018E00F0A42EFFE435F0CD89F0A42DFEE435F079
:10019E008067EF4E7005BD80D780C3EF8BF0A4ACA7
:1001AE00F0EE8BF0A42CFCE435F0F8EF8AF0A42CE2
:1001BE00E5F038FCE433CB8DF0A42CFCE5F03BF8F5
:1001CE00EE8AF0A42CFCE5F038F8E433CF89F0A4E5
:1001DE002CFCE5F038CF3400CE89F0A42FFFE5F0EB
:1001EE003EFEE433C98DF0A42EFEE5F039CD8AF043
:1001FE00A42FFFE5F03EFEE43DFD33D0E0FB5007BB
:10020E000BBB000F0203E5EC2CFCEF33FFEE33FECD
:06021E00ED33FD0203BDFB
:100224000203E5EC5D046005E8590470030203DB96
:100234001203A6580460F6EC4860F2EC7004FDFE6C
:10024400FF22C860DB2481C85009C39860025006AD
:100254000203E29850CAF582E9294B4A7005AB8241
:100264000203D175F0007C1A7880C3EF9BEE9AEDFF
:1002740099400DC3EF9BFFEE9AFEED99FDE842F025
:10028400DC23ACF0D0E0FFD0E0FED0E0FDAB822078
:10029400E7101BEB60BAEC2CFCEF33FFEE33FEED02
:1002A40033FD0203BDE803F830E705C0F075F00044
:1002B400EF2FFFEE33FEED33FD40B830E7C280AAE6
:1002C40074F8CC6480CCC86480C8F582046043C3ED
:1002D400EB9FF5F0EA9E42F0E99D42F0E89C45F080
:1002E40060305018E5825FFFE582F42B5582FB50A5
:1002F400210ABA001D09B90019088016E5825BFBC2
:10030400E582F42F5582FF50090EBE00050DBD0095
:10031400010CC3EB9FF5F0EA9E42F0E99D42F0E840
:0D0324009C45F06007CC4820E701B3EC22B7
:1003310075F020800E75F010800575F0087D007E47
:10034100007F003392D530D503120503EC33401002
:10035100EF33FFEE33FEED33FDEC33FCD5F0ED2250
:0E036100E5F0247EA2D513CC92E7CDCEFF228C
:10036F00EDD2E7CD33EC3392D524814006E4FFFE86
:10037F00FDFC22FCE4CFCECDCC24E0501174FF80E5
:10038F00EDC3CC13CCCD13CDCE13CECF13CF047082
:07039F00F030D5DE0205037A
:1012F5008F3F8E3E8D3D8C3C74FFFFFEFDFCAB3F6A
:10130500AA3EA93DA83CC3120511602C7F807E969C
:101315007D187C4BAB3FAA3EA93DA83C1202C46098
:101325000250157F807E967D187CCBAB3FAA3EA9E7
:101335003DA83C1202C45009AF3FAE3EAD3DAC3CAA
:1013450022AF3FAE3EAD3DAC3C12036F8F438E42A4
:101355008D418C40EC120331C8ECC8C9EDC9CAEE09
:10136500CACBEFCBAF3FAE3EAD3DAC3C120029E45E
:10137500FBFAF9F81202C4601A401874FF2543F508
:1013850043E54234FFF542E54134FFF541E540349C
:10139500FFF540AF43AE42AD41AC40EC1203312204
:1003A600E9D2E7C933E833F892D5EDD2E7CD33EC9D
:0703B60033FC5002B2D52216
:1003BD00EC30E7100FBF000C0EBE00080DBD0004A1
:1003CD000BEB6014A2D5EB13FCED92E7FD2274FF4D
:1003DD00FCFDFEFF22E480F8A2D574FF13FC7D80A6
:0303ED00E480EFBA
:030000000217F4F0
:0C17F400787FE4F6D8FD75819602183B62
:1003F000BB010689828A83E0225002E722BBFE020B
:09040000E32289828A83E493223D
:10040900BB010CE58229F582E5833AF583E02250A8
:1004190006E92582F8E622BBFE06E92582F8E222F2
:0D042900E58229F582E5833AF583E493220C
:10043600BB010689828A83F0225002F722BBFE01A5
:02044600F3229F
:10044800F8BB010DE58229F582E5833AF583E8F0EA
:10045800225006E92582C8F622BBFE05E92582C896
:02046800F2227E
:10046A00C2D5EC30E709B2D5E4C39DFDE49CFCEEAD
:10047A0030E715B2D5E4C39FFFE49EFE120644C3DB
:10048A00E49DFDE49CFC800312064430D507C3E4D6
:06049A009FFFE49EFE221C
:1004A000BB010A89828A83E0F5F0A3E02250068727
:1004B000F009E71922BBFE07E3F5F009E3192289E9
:0B04C000828A83E493F5F0740193221C
:1004CB00BB010789828A83020699500B09C5F02765
:1004DB00F7C5F01937F722BBFE0D09F8E325F0F34A
:1004EB00C5F019E338F322F889828A8374019325C6
:0804FB00F0C5F0F8E49338228B
:0E050300C3E49FFFE49EFEE49DFDE49CFC2209
:10051100EB9FF5F0EA9E42F0E99D42F0E89C45F040
:0105210022B7
:10052200E8600FEFC333FFEE33FEED33FDEC33FC37
:03053200D8F122DB
:10053500BB010789828A830206BB5005E9F80206DA
:10054500AFBBFE05E9F80206C789828A830206D396
:10055500BB010789828A8302059B5005E9F80205DC
:0A0565008FBBFE05E9F8020719221A
:10056F00BB010789828A830206F05005E9F802066B
:10057F00E3BBFE05E9F80206FC89828A83020709BC
:0C058F00ECF608EDF608EEF608EFF62298
:0C059B00ECF0A3EDF0A3EEF0A3EFF022D3
:1005A700A8828583F0D083D0821205BE1205BE12C1
:1005B70005BE1205BEE473E493A3C583C5F0C583E6
:1005C700C8C582C8F0A3C583C5F0C583C8C582C89E
:0105D7002201
:1005D800BB010789828A830205A75005E9F802074B
:0A05E80025BBFE05E9F802073E22DC
:1005F200D083D082F8E4937012740193700DA3A398
:1006020093F8740193F5828883E4737402936860AB
:06061200EFA3A3A380DFAB
:101E31008B378A388939E4F53FF540E53E153EAEEA
:101E41003D7002153D4E6033AB3AAA3BA93C1203EB
:101E5100F0FFAB37AA38A9390540E540AC3F700225
:101E6100053F14F5828C83EF120448EF60CD7401B5
:101E7100253CF53CE4353BF53B80C0AB37AA38A99E
:021E8100392204
:10061800EF4E6012EF60010EEDBB010B89828A83F9
:10062800F0A3DFFCDEFA2289F05007F709DFFCA906
:0C063800F022BBFEFCF309DFFCA9F0225D
:101800000220B6E493A3F8E493A34003F68001F228
:1018100008DFF48029E493A3F85407240CC8C333E9
:10182000C4540F4420C8834004F456800146F6DFB8
:10183000E4800B01020408102040809020C1E47E67
:10184000019360BCA3FF543F30E509541FFEE493AD
:10185000A360010ECF54C025E060A840B8E493A374
:10186000FAE493A3F8E493A3C8C582C8CAC583CA9F
:10187000F0A3C8C582C8CAC583CADFE9DEE780BE57
:0120CA000015
:10064400BC000BBE0029EF8DF084FFADF022E4CC9A
:10065400F875F008EF2FFFEE33FEEC33FCEE9DEC63
:10066400984005FCEE9DFE0FD5F0E9E4CEFD22EDA9
:10067400F8F5F0EE8420D21CFEADF075F008EF2FF3
:10068400FFED33FD4007985006D5F0F222C398FDE4
:050694000FD5F0EA2281
:10069900C5F0F8A3E028F0C5F0F8E58215827002EC
:0606A9001583E038F02289
:0C06AF00E6FC08E6FD08E6FE08E6FF2277
:0C06BB00E0FCA3E0FDA3E0FEA3E0FF22B2
:0C06C700E2FC08E2FD08E2FE08E2FF226F
:1006D300E493FC740193FD740293FE740393FF226D
:0D06E300E6FB08E6F908E6FA08E6CBF82287
:0C06F000E0F8A3E0F9A3E0FAA3E0FB228D
:0D06FC00E2FB08E2F908E2FA08E2CBF8227E
:10070900E493F8740193F9740293FA740393FB2246
:0C071900ECF208EDF208EEF208EFF2221C
:10072500D083D082E493F608740193F6087402939B
:09073500F608740393F6740473D2
:10073E00D083D082E493F208740193F2087402938A
:09074E00F208740393F2740473C1
:00000001FF
